:1000000000308A00B12800000A108A100A11820705
:100010000A340D3400340A108A100A1182072A3477
:100020002A342A340A340D3400340A108A100A1192
:100030008207733465346E3473346F347234203411
:100040002534753420342D342034253475340A3465
:100050000D34003483168611831286110830F8009F
:10006000000000000000F8174428F813AA0C031839
:100070008615031C8611781744287813F80B362848
:1000800000000000000086151C308400840B462808
:10009000000000006400F81B3528781B3D28003460
:1000A000273084000008031966280130F800BF30AB
:1000B000F7006400F70B5928F80B57284A30F7006F
:1000C000F70B602800006400800B552800342B08D3
:1000D000F8012A0203186F282A08F7007B28F70185
:1000E0000830AC00AA0DF70D2B0877020318F700B3
:1000F000F80DAC0B7228003478082808AA00643088
:10010000AB0067207708A80078083030031D8F28DF
:10011000A91C9628A9199628291A20309228A911D5
:1001200029122914F8077808AA002A202808AA000A
:100130000A30AB0067207708A80078083030031D2C
:10014000A728A919AB28291CAB28291A2030F807A1
:100150007808AA002A203030A8072808AA002A20F8
:10016000003484011F308305603083168F008611B0
:100170008312861583161F129F121B0880399B005D
:1001800007309C001F129F121B0880397F389B008C
:100190001F1383121F179F1783169F1383121F1499
:1001A00094128316061186140616353083129400B5
:1001B0004030831694000108C73908388100831243
:1001C00090010030F8009200003083169200073052
:1001D0009C00050864000230F700F70BED280000D2
:1001E00000001C0883120D1383169D010830831232
:1001F000A100A200A7012708042000380319042940
:10020000A70AAA002A20FB286430A7005020A701D3
:1002100027080B20003803191129A70AAA002A2051
:1002200008296430A7005020A6012608063C031CBC
:100230005129260DF700F70DF70DF830F7051F08C7
:10024000C73977049F006430A70050201F151F197D
:1002500027291E08A500A70127081520A70AF700CF
:10026000AA002A2007302702031D2C292608A800EF
:100270001B30A9007C202030AA002A202D30AA00A3
:100280002A202030AA002A202508A8001B30A90017
:100290007C200A30AA002A200D30AA002A20A60AB3
:1002A0001529A3010030F8001F08C73978049F0002
:1002B000A40164000230F700F70B5C290000000085
:1002C0001F151F1961291E08A5000830F8001F0816
:1002D000C73978049F002508453C031C7829250868
:1002E000323C0318772922080139A4047829241400
:1002F0001F151F1979291E08A5001030F8001F08C6
:10030000C73978049F002508453C031C902925081F
:10031000323C03188F2922080239A4049029A4141E
:100320001F151F1991291E08A5001830F8001F0875
:10033000C73978049F002508453C031CA8292508D7
:10034000323C0318A72922080439A404A82924153B
:100350001F151F19A9291E08A5002030F8001F0825
:10036000C73978049F002508453C031CC02925088F
:10037000323C0318BF2922080839A404C029A41557
:100380001F151F19C1291E08A5002830F8001F08D5
:10039000C73978049F002508453C031CD829250847
:1003A000323C0318D72922081039A404D82924166E
:1003B0001F151F19D9291E08A5003030F8001F0885
:1003C000C73978049F002508453C031CF0292508FF
:1003D000323C0318EF2922082039A404F029A4167E
:1003E0001F151F19F1291E08A5002508453C031CEF
:1003F000022A2508323C0318012A22084039A404A5
:10040000022A24172408A200831606148312061851
:100410000E2A230F0C2A0D2AA30A0F2AA301230850
:100420000A3C031CA417A40924089300831614187B
:0C0430001B2A8312162A83125229630033
:04400E00383FFC3FFC
:00000001FF
